:0200000480007A
:100000006F008004732F2034930F80006308FF0378
:10001000930F90006304FF03930FB0006300FF038E
:10002000130F000063040F0067000F00732F2034CC
:1000300063540F006F00400093E19153171F0000BD
:1000400023223FFC6FF09FFF93000000130100008C
:10005000930100001302000093020000130300004C
:100060009303000013040000930400001305000034
:10007000930500001306000093060000130700001C
:100080009307000013080000930800001309000004
:1000900093090000130A0000930A0000130B0000EC
:1000A000930B0000130C0000930C0000130D0000D4
:1000B000930D0000130E0000930E0000130F0000BC
:1000C000930F0000732540F16310050097020000B4
:1000D000938202017390523073500018970200000F
:1000E00093824202739052309B021000939252030B
:1000F0009382F2FF7390023B9302F0017390023AF5
:100100007350403097020000938242017390523046
:10011000735020307350303093010000970200007C
:10012000938282EE73905230130510001315F5017F
:10013000635C05000F00F00F930110009308D005D9
:10014000130500007300000093020000638A0200A0
:1001500073905210B7B200009B82921073902230BD
:100160007350003097020000938242017390123462
:10017000732540F17300203093000000130100004C
:10018000338720409303000093012000631E774AC9
:1001900093001000130110003387204093030000E8
:1001A000930130006312774A93003000130170000E
:1001B000338720409303C0FF9301400063167748C4
:1001C000930000003781FFFF33872040B783000092
:1001D00093015000631A7746B700008013010000B6
:1001E00033872040B703008093016000631E77448B
:1001F000B70000803781FFFF33872040B78300803E
:10020000930170006312774493000000378100006F
:100210001B01F1FF33872040B783FFFF9B8313004F
:100220009301800063127742B70000809B80F0FF4B
:100230001301000033872040B70300809B83F3FF46
:100240009301900063127740B70000809B80F0FF1D
:10025000378100001B01F1FF33872040B783FF7F08
:100260009301A0006312773EB70000803781000041
:100270001B01F1FF33872040B703FFFF9B83F3FF90
:100280009393F300938313009301B000631E773AB6
:10029000B70000809B80F0FF3781FFFF338720404D
:1002A000B70301009B8313009393F3009383F3FF41
:1002B0009301C000631A7738930000001301F0FF28
:1002C00033872040930310009301D000631E7736DC
:1002D0009300F0FF13011000338720409303E0FFE9
:1002E0009301E000631277369300F0FF1301F0FFF3
:1002F00033872040930300009301F00063167734A6
:100300009300D0001301B000B3802040930320007D
:1003100093010001639A70329300E0001301B00072
:10032000338120409303300093011001631E71302C
:100330009300D000B380104093030000930120018C
:1003400063947030130200009300D0001301B000DA
:10035000338720401303070013021200930220008A
:10036000E31452FE9303200093013001631E732CAB
:10037000130200009300E0001301B0003387204017
:100380001300000013030700130212009302200061
:10039000E31252FE93033000930140016316732A67
:1003A000130200009300F0001301B00033872040D7
:1003B00013000000130000001303070013021200D3
:1003C00093022000E31052FE93034000930150017A
:1003D000631C7326130200009300D0001301B000C9
:1003E000338720401302120093022000E31652FECE
:1003F0009303200093016001631877241302000027
:100400009300E0001301B000130000003387204088
:100410001302120093022000E31452FE93033000F3
:100420009301700163127722130200009300F00021
:100430001301B000130000001300000033872040B8
:100440001302120093022000E31252FE93034000B5
:1004500093018001631A771E130200009300D000FD
:10046000130000001301B000338720401302120074
:1004700093022000E31452FE9303200093019001A5
:100480006314771C130200009300E00013000000C7
:100490001301B00013000000338720401302120044
:1004A00093022000E31252FE930330009301A00157
:1004B000631C7718130200009300F0001300000083
:1004C000130000001301B000338720401302120014
:1004D00093022000E31252FE930340009301B00107
:1004E00063147716130200001301B0009300D000CC
:1004F000338720401302120093022000E31652FEBD
:10050000930320009301C0016310771413020000CD
:100510001301B0009300E000130000003387204077
:100520001302120093022000E31452FE93033000E2
:100530009301D001631A7710130200001301B00079
:100540009300F000130000001300000033872040E8
:100550001302120093022000E31252FE93034000A4
:100560009301E0016312770E130200001301B00043
:10057000130000009300D0003387204013021200C4
:1005800093022000E31452FE930320009301F00134
:10059000631C770A130200001301B000130000006F
:1005A0009300E00013000000338720401302120084
:1005B00093022000E31252FE9303300093010002E5
:1005C00063147708130200001301B0001300000049
:1005D000130000009300F000338720401302120044
:1005E00093022000E31252FE930340009301100295
:1005F000631C7704930010FF330110409303F00055
:1006000093012002631271049300000233810040C1
:10061000930300029301300263187102B30000409B
:100620009303000093014002639070029300000165
:100630001301E00133802040930300009301500236
:1006400063147000631030020F00F00F638001002C
:100650009391110093E111009308D00513850100D7
:10066000730000000F00F00F930110009308D005F5
:0C0670001305000073000000731000C0B0
:1010000000000000000000000000000000000000E0
:1010100000000000000000000000000000000000D0
:1010200000000000000000000000000000000000C0
:1010300000000000000000000000000000000000B0
:081040000000000000000000A8
:040000058000000077
:00000001FF
